S00C0000446F6F722E7372656384
S11300000C9435000C9422070C945D000C945D0054
S11300100C945D000C945D000C945D000C945D00E8
S11300200C945D000C945D000C945D000C945D00D8
S11300300C945D000C945F000C945D000C945D00C6
S11300400C945D000C945D000C945D000C945D00B8
S11300500C945D000C945D000C945D000C945D00A8
S11300600C945D000C945D00DA0711241FBECFEFE1
S1130070D4E0DEBFCDBF11E0A0E0B1E0EEE0F3E1FB
S113008002C005900D92A438B107D9F721E0A4E885
S1130090B1E001C01D92AB3BB207E1F710E0CAE644
S11300A0D0E004C02297FE010E948109C836D1071E
S11300B0C9F70E9421030C9485090C9400001F9237
S11300C00F920FB60F9211242F923F924F925F928C
S11300D06F927F928F929F92AF92BF92CF92DF9254
S11300E0EF92FF920F931F932F933F934F935F933E
S11300F06F937F938F939F93AF93BF93CF93DF932C
S1130100EF93FF93D0918801DD2309F40BC220E023
S113011030E0A9016091A1017091A2018091A30135
S11301209091A4010E9465088111FCC020E030E098
S1130130A9016091A5017091A6018091A7019091F8
S1130140A8010E9465088111F0C020E030E0A901F7
S11301506091A9017091AA018091AB019091AC01C9
S11301600E9465088111E4C0C091B9012C2F30E0D0
S11301702F5F3F4F8D2F90E02817390714F4CF5F7E
S113018001C0C0E0C093B901BB24B394D0E00F2EEA
S1130190F4EBCF2ED12CF02D0F2EFBE96F2EF1E0D6
S11301A07F2EF02D6C0E7D1E01C0B3941B2D1150BB
S11301B0E12EF12C9E01F701EE0FFF1FEE0DFF1D46
S11301C0EE0FFF1FE857FE4FEC0FFD1F818190E0FB
S11301D0113009F120F0123009F057C039C048B588
S11301E09701220F331F220F331F890108571E4F17
S11301F0841B9109F301608170E00E944B098827F8
S113020077FD8095982F0E949708F801618F728F6F
S1130210838F948F5DC0F60140819701220F331FB5
S1130220220F331F890108571E4F841B9109F301C4
S1130230608170E00E944B09882777FD8095982F94
S11302400E949708F801618F728F838F948F42C048
S11302504091B300E701CC0FDD1FCC0FDD1FC85761
S1130260DE4F841B9109F901E857FE4F638970E062
S11302700E944B09882777FD8095982F0E94970844
S1130280698F7A8F8B8F9C8F28C09701220F331F21
S1130290220F331F0F2EF8E88F2EF1E09F2EF02D42
S11302A0820E931EF301608170E00E944B0988273F
S11302B077FD8095982F0E949708F401618F728FC3
S11302C0838F948F113031F018F01230C9F405C0C7
S11302D068B510C1F60160810DC16091B300E701FA
S11302E0CC0FDD1FCC0FDD1FC857DE4F70E080E060
S11302F090E00E9495086DA37EA38FA398A712C1D6
S1130300F701EE0FFF1FEE0FFF1FE857FE4F15A278
S113031016A217A210A6F2E0FB1508F046CF02C100
S1130320839414C08824839405C08824839402C0D1
S11303308824839409EB11E00F2EF4EBAF2EB12C3B
S1130340F02D0F2EF3EB2F2E312CF02D982C9A94A8
S1130350C92DD0E0FE01EE0FFF1FEE0FFF1FE8577F
S1130360FE4FC18CD28CE38CF48C20E030E0A901E8
S1130370C701B6010E944709181664F5FE01EE0F85
S1130380FF1FEE0FFF1FE857FE4F25A136A147A11F
S113039050A5C701B6010E9401082B013C01F801D8
S11303A08081FE01EE0FFF1FEC0FFD1FEE0FFF1FFC
S11303B0E857FE4FE80FF11D618170E080E090E0A6
S11303C00E9497089B01AC01C301B2010E94650819
S11303D01816B4F520E030E0A901C701B6010E9467
S11303E0650888230CF059C0FE01EE0FFF1FEE0FC5
S11303F0FF1FE857FE4F25A136A147A150A5C7010D
S1130400B6010E9401082B013C01F8018081FE0124
S1130410EE0FFF1FEC0FFD1FEE0FFF1FE857FE4FFF
S1130420E80FF11D618170E080E090E00E94970880
S11304309B01AC01C301B2010E94470988236CF1FE
S1130440CC0FDD1FCC0FDD1FC857DE4F2DA13EA101
S11304504FA158A5C701B6010E940108262F372FC6
S1130460462F572F682F792F4DA35EA36FA378A72C
S1130470622F732F0E946908F1E09F1641F09F16C6
S113048020F082E0981231C005C068BD49CFF50163
S1130490608346CF6093B30045C0F8018081FE01BC
S11304A0EE0FFF1FEC0FFD1FEE0FFF1FE857FE4F6F
S11304B0E80FF11D8181F1E09F1641F09F1620F0B5
S11304C092E0991208C005C088BD05C0F50180837B
S11304D002C0F1018083CC0FDD1FCC0FDD1FC85794
S11304E0DE4F198E1A8E1B8E1C8EF2E0F81508F062
S11304F017CF18C0C701880F991F880F991F0F2E97
S1130500F8E8EF2EF1E0FF2EF02DE80EF91E70E072
S113051080E090E00E949508F70165A376A387A385
S113052090A743CEFF91EF91DF91CF91BF91AF910F
S11305309F918F917F916F915F914F913F912F91F7
S11305401F910F91FF90EF90DF90CF90BF90AF90ED
S11305509F908F907F906F905F904F903F902F90DF
S11305600F900FBE0F901F901895CF93DF93789440
S113057081E88093C4001092C00088E08093C10099
S113058086E08093C200A1E0B1E095E5E0ECF0E004
S1130590C6ECD0E0808185FFFDCF98839D919111B9
S11305A0F9CFE0ECF0E0808185FFFDCF8DE0809312
S11305B0C600E0ECF0E0808185FFFDCF8AE0809307
S11305C0C600DF91CF91089560FF04C08FEF809340
S11305D0B30002C01092B30061FF04C08FEF809398
S11305E0B40002C01092B40062FF03C08FEF88BD54
S11305F0089518BC0895CF93DF93FB01908199234C
S113060069F0DB011196E0ECF0E0C6ECD0E080810B
S113061085FFFDCF98839D919111F9CFE0ECF0E037
S1130620808185FFFDCF8DE08093C600E0ECF0E093
S1130630808185FFFDCF8AE08093C600DF91CF9152
S11306400895CF93DF9300D000D01F92CDB7DEB7CB
S1130650789464E088E891E00E94E4026BE071E041
S11306608AEB91E00E94FB022FE73AE186E02150F9
S113067030408040E1F700C0000062E088E891E08B
S11306800E94E40260E171E08AEB91E00E94FB02C7
S11306909FE7AAE1B6E09150A040B040E1F700C066
S11306A0000061E088E891E00E94E40266E171E004
S11306B08AEB91E00E94FB022FE73AE186E02150A9
S11306C030408040E1F700C0000067E088E891E036
S11306D00E94E4026CE171E08AEB91E00E94FB026B
S11306E09FE7AAE1B6E09150A040B040E1F700C016
S11306F00000299A60E088E891E00E94E402312C2D
S113070045E851E01FEF0F2EF9E8EF2EF1E0FF2E40
S1130710F02D0F2EF5E98F2EF1E09F2EF02D0F2EE8
S1130720FBE96F2EF1E07F2EF02D0F2EFAE02F2E35
S1130730F02D0F2EF8E84F2EF1E05F2EF02DAA24B5
S1130740A3940F2EF9EBCF2EF1E0DF2EF02DE0EC89
S1130750F0E00F2EFDE0BF2EF02D3982012FDA01DB
S11307608C910C938C3009F4F9C038F5853009F478
S113077082C090F4823009F458C038F4882309F414
S113078046C0813009F0EAC149C0833009F45CC035
S1130790843009F0E3C161C0883009F496C038F4AC
S11307A0863009F476C0873009F0D8C180C08A3019
S11307B009F4A9C008F0B6C097C0823109F43AC15F
S11307C090F48F3009F4F7C038F48D3009F4D5C0B3
S11307D08E3009F0C3C1E0C0803109F40DC181310C
S11307E009F0BCC118C1853109F47CC138F48331E6
S11307F009F42FC1843109F0B1C166C1873109F40C
S11308008DC108F47DC18F3F09F0A8C14EC2B981E2
S1130810BF3F09F44AC2BF5FB98347C2298122237B
S113082009F443C22150298340C284B58F7D84BD1D
S1130830A0EBB0E08C918F758C935D98559A5B9882
S1130840539A2B98239A31C284B5806284BDA0EB5D
S1130850B0E08C91806A8C9328C2D7011C93AFE8D6
S1130860B1E01C92D4011C92D3012C92D201AC921F
S1130870D6011C921AC2D7011C92AFE8B1E01C93B6
S1130880D4011C92D3012C92D201AC92D6011C92B9
S11308900CC2D7011C92AFE8B1E01C92D4011C93A6
S11308A0D3012C92D201AC92D6011C92FEC1D70185
S11308B01C93AFE8B1E01C93D4011C93D3012C9298
S11308C0D201AC92D6011C92F0C1D7011C9380E4F2
S11308D0AFE8B1E08C93D4011C92D3012C92D201E5
S11308E0AC92D6011C92E1C1D7011C92AFE8B1E0F1
S11308F01C9380E4D4018C93D3012C92D201AC924A
S1130900D6011C92D2C180E4D7018C93AFE8B1E048
S11309101C92D4011C93D3012C92D201AC92D60127
S11309201C92C3C1D7011C93AFE8B1E01C93D4015E
S11309301C932981D3012C93AAE8B1E01C92A0E96D
S1130940B1E01C92A6E9B1E01C92ACE9B1E02C93B1
S113095082E0D2018C93D6011C92A7C1D7011C93CB
S113096020E8AFE8B1E02C93D4011C92D3012C927F
S1130970D201AC92D6011C9298C1D7011C92AFE867
S1130980B1E01C9320E8D4012C93D3012C92D20122
S1130990AC92D6011C9289C120E8D7012C93AFE810
S11309A0B1E01C92D4011C93D3012C92D201AC92DD
S11309B0D6011C927AC18091B3009091B40028B5FD
S11309C0D7012C93AFE8B1E09C93D4018C93298197
S11309D0D3012C93AAE8B1E01C92A0E9B1E01C92E7
S11309E0A6E9B1E01C92ACE9B1E02C9382E0D2011B
S11309F08C93D6011C9259C1D7011C9320ECAFE80B
S1130A00B1E02C93D4011C92D3012C92D201AC926C
S1130A10D6011C924AC1D7011C92AFE8B1E01C93E5
S1130A2020ECD4012C93D3012C92D201AC92D601A8
S1130A301C923BC120ECD7012C93AFE8B1E01C928F
S1130A40D4011C93D3012C92D201AC92D6011C92F6
S1130A502CC1D7011C93AFE8B1E01C92D4011C92C5
S1130A60D3011C93AAE8B1E01C93A0E9B1E01C9364
S1130A70A6E9B1E01C92ACE9B1E01C9310928B01A1
S1130A80109391011092970110939D0110928C0183
S1130A90109392011093980110939E0110928D016E
S1130AA0109293011093990110939F0110938E015A
S1130AB01092940110939A011093A00186E0D20140
S1130AC08C93D6011C92F1C0D7011C93AFE8B1E01E
S1130AD01C93D4011C92D3012C92D201AC92D60166
S1130AE01C92E3C0D7011C92AFE8B1E01C93D4017F
S1130AF01C93D3012C92D201AC92D6011C92D5C086
S1130B00D7011C93AFE8B1E01C92D4011C93D3012C
S1130B102C92D201AC92D6011C92C7C0D7011C9270
S1130B20AFE8B1E01C9320E1D4012C9329E1D30177
S1130B302C93AAE8B1E01C922AEAA0E9B1E02C9334
S1130B4020E1A6E9B1E02C938FE0ACE9B1E08C930D
S1130B5082E0D2018C93D6011C92A7C0282F30E0EA
S1130B603B832A83808185FFFDCF80E3A6ECB0E040
S1130B708C9360E070E0CB01969587959695879568
S1130B80969587959C01220F331F880F991F880F14
S1130B90991F880F991F820F931F681B790B605D43
S1130BA0808185FFFDCFA6ECB0E06C932A813B8168
S1130BB03695279536952795ABE7B4E10E945F09F2
S1130BC096958795805D908195FFFDCFA6ECB0E06A
S1130BD08C932A813B81ADECBCEC0E945F09969515
S1130BE0879596958795969587959D838C839C018B
S1130BF00E945F0996958795969587959695879512
S1130C009C01220F331F880F991F880F991F880F8B
S1130C10991F820F931F2C813D81281B390BC90119
S1130C20805D908195FFFDCFA6ECB0E08C932A8186
S1130C303B81ADECBCEC0E945F0996958795969537
S1130C408795969587959C01220F331F880F991FCE
S1130C50880F991F880F991F820F931F2A813B8148
S1130C60281B390BC901805D908195FFFDCFA6EC4F
S1130C70B0E08C93A3E6B1E090E29D01808185FF12
S1130C80FDCFA6ECB0E09C93D9019D919D019111FB
S1130C90F5CF808185FFFDCFA6ECB0E0BC928081CA
S1130CA085FFFDCFA6ECB0E02C9200B605FE2DC06A
S1130CB0311058C0D7011C93AFE8B1E01C92D401A5
S1130CC01C9284E6D3018C93D201AC92D6011C927F
S1130CD0ADE6B1E094E59D01808185FFFDCFA6ECF2
S1130CE0B0E09C93D9019D919D019111F5CF808134
S1130CF085FFFDCFA6ECB0E0BC92808185FFFDCFDF
S1130D00A6ECB0E02C923A2C2DC0B1E03B122AC0E4
S1130D10A7E7B1E094E59D01808185FFFDCFA6ECB6
S1130D20B0E09C93D9019D919D019111F5CF8081F3
S1130D3085FFFDCFA6ECB0E0BC92808185FFFDCF9E
S1130D40A6ECB0E02C92D7011C92AFE8B1E01C9362
S1130D50D4011C9282E3D3018C93D201AC92D601CC
S1130D601C92312C87E893E10197F1F700C0000051
S1130D7029989FEDAAE0B6E09150A040B040E1F779
S1130D8000C00000299AEBCC559A539A239AFC018F
S1130D90108211AA81E084BD94E095BD16BC109226
S1130DA0800092E09093810010928500109284005C
S1130DB01092B600E0EBF0E0808395E09093B100F0
S1130DC01092B20010926E0080936F001092700027
S1130DD084B5806284BD8081806A808318BC10924F
S1130DE0B4001092B300089520E030E080E061E0A8
S1130DF070E04A9BFECFEFE9FFE03197F1F700C0C6
S1130E0000004A9B08C0AB01022E02C0440F551FCC
S1130E100A94E2F7842B4A990FC008C04A9B06C083
S1130E20F5E8FA95F1F700009150C1F72F5F3F4FB5
S1130E3028303105F1F6089545E84A95F1F70000A8
S1130E4091E3ECCF1F920F920FB60F9211242F93C0
S1130E503F934F935F936F937F938F939F93AF933E
S1130E60BF93CF93EF93FF93289A4A9979C08FE168
S1130E709EE40197F1F700C000004A9971C04A9BB3
S1130E80FECF4A99FECF80E090E060E041E050E080
S1130E904A9BFECFEFE9FFE03197F1F700C0000075
S1130EA04A9B08C09A01082E02C0220F331F0A94DD
S1130EB0E2F7622B4A9966C008C04A9B06C0F5E86F
S1130EC0FA95F1F700002150C1F701968830910599
S1130ED0F9F6611139C080E090E041E050E04A9BAE
S1130EE0FECFEFE9FFE03197F1F700C000004A9B25
S1130EF008C09A01082E02C0220F331F0A94E2F799
S1130F00622B4A9939C008C04A9B06C0F5E8FA9595
S1130F10F1F700002150C1F7019688309105F9F6E8
S1130F206F3E91F484E891E00E94F406C82F84E8AF
S1130F3091E00E94F406282F30E02C0F311D2F3F42
S1130F40310511F4CF3F51F42FE734E88EE12150FD
S1130F5030408040E1F700C000000BC0CE3F39F4C0
S1130F60E7E8F3E13197F1F700C0000002C0C09355
S1130F7085012898E09A0CC0F5E8FA95F1F700008D
S1130F8021E3C2CF25E82A95F1F7000021E395CFAC
S1130F90FF91EF91CF91BF91AF919F918F917F91ED
S1130FA06F915F914F913F912F910F900FBE0F90D2
S1130FB01F9018958AEB91E00E94B50288E891E0B1
S1130FC00E94C406209A219A2898299856985E98D7
S1130FD057985F9810BE10927B0083E080937F0047
S1130FE0209A219A2898299852985A988FEF80939A
S1130FF0850182E08093690081E08DBB1CBA08956D
S11310005058BB27AA270ED008C1F9D030F0FED023
S113101020F031F49F3F11F41EF4EEC00EF4E0957D
S1131020E7FBE4C0E92F0AD180F3BA17620773071C
S11310308407950718F071F49EF522C10EF4E0952B
S11310400B2EBA2FA02D0B01B90190010C01CA017E
S1131050A0011124FF27591B99F0593F50F4503E29
S113106068F11A16F040A22F232F342F4427585F1B
S1131070F3CF469537952795A795F0405395C9F733
S11310807EF41F16BA0B620B730B840BBAF09150EB
S1131090A1F0FF0FBB1F661F771F881FC2F70EC08A
S11310A0BA0F621F731F841F48F48795779567955D
S11310B0B795F7959E3F08F0B3CF9395880F08F046
S11310C09927EE0F9795879508956CD008F481E0E1
S11310D00895BCD088F09F5790F0B92F9927B75145
S11310E0A0F0D1F0660F771F881F991F1AF0BA95E8
S11310F0C9F712C0B13081F0C3D0B1E00895C0C0C7
S1131100672F782F8827B85F39F0B93FCCF38695DD
S113111077956795B395D9F73EF49095809570953A
S113112061957F4F8F4F9F4F0895E89409C097FBB7
S11311303EF490958095709561957F4F8F4F9F4FAA
S11311409923A9F0F92F96E9BB279395F6958795EE
S113115077956795B795F111F8CFFAF4BB0F11F4B1
S113116060FF1BC06F5F7F4F8F4F9F4F16C0882358
S113117011F096E911C0772321F09EE8872F762F8E
S113118005C0662371F096E8862F70E060E02AF0CF
S11311909A95660F771F881FDAF7880F96958795BB
S11311A097F90895990F0008550FAA0BE0E8FEEF90
S11311B016161706E807F907C0F012161306E40717
S11311C0F50798F0621B730B840B950B39F40A2610
S11311D061F0232B242B252B21F408950A2609F4EE
S11311E0A140A6958FEF811D811D089597F99F67F2
S11311F080E870E060E008959FEF80EC089500249B
S11312000A941616170618060906089500240A9467
S113121012161306140605060895092E0394000CED
S113122011F4882352F0BB0F40F4BF2B11F460FF7C
S113123004C06F5F7F4F8F4F9F4F089557FD9058A5
S1131240440F551F59F05F3F71F04795880F97FB86
S1131250991F61F09F3F79F0879508951216130640
S11312601406551FF2CF4695F1DF08C0161617066F
S11312701806991FF1CF86957105610508940895A4
S1131280E894BB2766277727CB0197F908958ADF6F
S113129008F48FEF089597FB072E16F4009407D0F7
S11312A077FD09D00E946B0907FC05D03EF49095A8
S11312B081959F4F0895709561957F4F0895A29FE2
S11312C0B001B39FC001A39F01D0B29F700D811DD7
S11312D01124911D0895AA1BBB1B51E107C0AA1F2D
S11312E0BB1FA617B70710F0A61BB70B881F991FC3
S11312F05A95A9F780959095BC01CD010895EE0FFC
S1111300FF1F0590F491E02D0994F894FFCF9F
S113130E5561727420646F6E652100526F742100F2
S113131E4772FC6E2100426C61752100576569DFCE
S113132E2C20616C6C657320496E697469616C69FB
S113133E7365727421204861626520466572746912
S113134E6720756E642064616D6974206162207A11
S113135E756D204E6F726D616C6265747269656233
S113136E21002050726573736564210054FC722051
S113137E5A752E2E2E0054FC72204F6666656E2E04
S107138E2E2E0000FB
S9030000FC
